:03000000024714A0
:0C47140078FFE4F6D8FD75816102475B78
:101EA30020000A3C2E2E2E3E004950436F6E6E6575
:101EB30063745245510A004950436F6E6E656374F3
:101EC300000A49504E6F41434B210A003E432C56B2
:101ED3002C43432CC0E4E0EFF2E5F020D1E8EDEA37
:101EE300EEEC49500A003E432C4D41432C25303241
:101EF30062583A25303262583A25303262583A25D0
:101F0300303262583A25303262583A2530326258BC
:101F13002C4D414320E0E4F0E5F10A003E432C560A
:101F230045522C20332E3220EEF2202573202573C8
:101F33002CC2E5F0F1E8FF20495020ECEEE4F3EB8E
:101F4300FF0A004F637420323320323030390030BF
:101F5300383A35363A3338003E432C4C442C5052F1
:101F63004F473A20202020202020202020202020FE
:101F7300202020202020202020202020202020205E
:101F8300202020202020202020202020202020204E
:101F9300202020202020202020202020202020203E
:101FA30020202020202020202CC4E0F2E020EFF08D
:101FB300EEF8E8E2EAE828F4E0E9EB290A003E2A31
:101FC3002C312CCEF1EDEEE2EDFBE520EFE0F0E07D
:101FD300ECE5F2F0FB20F1E5F2E5E2EEE3EE20E8DA
:101FE300EDF2E5F0F4E5E9F1E00A003E412C413081
:101FF300312C2562752E2562752E2562752E25627C
:10200300752C495020E0E4F0E5F120E0E4E0EFF244
:10201300E5F0E00A003E412C4130322C2562752E5A
:102023002562752E2562752E2562752C495020E098
:10203300E4F0E5F120EEF1ED2E20F1E5F0E2E5F03C
:10204300E00A003E412C4130332C2562752E256277
:10205300752E2562752E2562752C495020E0E4F01B
:10206300E5F120F0E5E72E20F1E5F0E2E5F0E00A06
:10207300003E412C4130342C2562752E2562752E8D
:102083002562752E2562752CCCE0F1EAE020F1E59E
:10209300F2E80A003E412C4130352C2562752E258D
:1020A30062752E2562752E2562752CD8EBFEE70A24
:1020B300003E2A2C312CC4EEEF2E20EFE0F0E0ECB2
:1020C300E5F2F0FB20F1E5F2E5E2EEE3EE20E8EDE8
:1020D300F2E5F0F4E5E9F1E00A003E422C53303139
:1020E3002C2562752CC6E4E0F2FC20E7E0EFF0EE6D
:1020F300F1E020F1EEE5E4E8EDE5EDE8FF20EEF2B6
:1021030020F1E5F0E2E5F0E00A003E422C533032E4
:102113002C2562752CCEE1ECE5ED20F120F1E5F004
:10212300E2E5F0EEEC20E1E5E720EAE2E8F2E0EDBB
:10213300F6E8E90A003E422C5330332C2562752C15
:10214300CFE5F0E5E7E0EFF3F1EA20EFF0E820EF89
:10215300EEF2E5F0E520F1E2FFE7E820F120F1E51A
:10216300F0E2E5F0EEEC0A003E422C5330352C252C
:1021730062752CCAE0EDE0EB20F8E8F0EEEAEEE25F
:10218300E5F8E0F2E5EBFCEDEEE3EE20EEE1ECE565
:10219300EDE00A003E532C5330362C253032625882
:1021A3002530326258253032625825303262582544
:1021B3003032625825303262582C4D414320E0E4DE
:1021C300F0E5F120F8E8F0EEEAEEE2E5F8E0F2E51A
:1021D300EBFCEDEEE3EE20EEE1ECE5EDE00A003E94
:1021E300454E440A000A44756D7058202020202073
:1021F3003030203031203032203033203034203022
:1022030035203036203037203038203039203041E7
:1022130020304220304320304420304520304600D7
:102223000A3A003A20000A000A44756D70442020DF
:102233002020203030203031203032203033203005
:1022430034203035203036203037203038203039B4
:10225300203041203042203043203044203045207C
:10226300304600457272206B6579005264206565C3
:1022730070726F6D0A005264204D454D0A0052641E
:1022830020436F64650A00577269746520436F6465
:10229300650A0044656275674950204F4E0A004441
:1022A300656275674950204F46460A00446562756A
:1022B3006755736572204F6E0A00446562756755F2
:1022C300736572204F46460A0044656275674D7315
:1022D30067204F6E0A0044656275674D7367204F30
:1022E30046460A00436F6E666967206C6F636B2115
:1022F3000A00577220656570726F6D0A0020536182
:10230300766520656570726F6D210A0045727220D3
:102313004D414321004C6F61643E3E002A00CEF8DC
:10232300E8E1EAE00A00202D202575282575290A11
:10233300003C4130313D003C4130323D003C4130B6
:10234300333D003C4130343D003C4130353D003CA1
:1023530021003C5330313D003C5330323D003C536F
:1023630030333D003C5330353D003C5330363D0067
:06514600015E00015C00A7
:10510900C28E438910758BFF758DB7D2ABD28E22B3
:03001B0002468416
:10468400C0E0C083C082C0D0C28E758BFF758DB769
:1046940020060675A61E75A6E1055CD202E55E60DD
:1046A40002055EE55DD394014002155D0561E56197
:1046B400540F7048D20EE561543F7012D200906ED0
:1046C400C7E0600A04F0E0D394B44002D206906ECE
:1046D400C0E0600204F090693EE0600214F0906E65
:1046E400C8E0D394014003E014F0300502055FE50F
:1046F40060D394644004D20680020560E55BD394E1
:10470400014002155BD28ED0D0D082D083D0E0326B
:1011BE00C291C290D2B5C20B7D027C007F07125045
:1011CE00AA8F26E526646060097D017F6012504576
:1011DE00D20BE4FDFC7F0B1250AA8F26E52630E6DB
:1011EE00097D04E4FF125069D20B7D017C007F075C
:1011FE001250AA8F26E5267008FD7FFF125045D2A9
:10120E000B300B03126000C288C2A8C2AA758900F7
:10121E00124AC0906B78E0B4FA06A3E064CE607B0D
:10122E00E4F52674702526F582E4346BF583E4F03C
:10123E000526E526B443EC906B7874FAF0A374CED1
:10124E00F0A374CCF0906B7E740AF0E4A3F0A304C8
:10125E00F0A3F0906B7474FFF0A3F0A3F0E4A3F08E
:10126E00906B8F740AF0E4F526E5262401FFE43333
:10127E00FE74702526F582E4346BF583E0FD125082
:10128E00210526E526C3944340DFE4F5A775A61E87
:10129E0075A6E1907FF0F0A3F080FE906B8374034F
:1012AE00F0A374CCF0E4906B82F0906EC5F0A3F0D6
:1012BE00124320C2B5123375C206124DA2D20BC212
:1012CE000DC20C906DB07408F0906AEE7424F0E4C8
:1012DE00A3F0906B78E0906AF0F0906B79E0906AF2
:1012EE00F1F0906B7AE0906AF2F0906B7BE0906A8E
:1012FE00F3F0906B7CE0906AF4F0906B7DE0906A76
:10130E00F5F0755D01E4906DB1F0C207C208C20937
:10131E00C20A124FFA200B19AF267E007D0312402F
:10132E008FE4FF12449C7E1E7FA3E4FBFDFC123D66
:10133E009C906EC7E060037401F0E490693EF0F596
:10134E005F906DAFF0F56012510975A70775A61E77
:10135E0075A6E1D2AFE4F56090693EE07003122607
:10136E00CF906EC8E06401701D9080007410F090F4
:10137E0080A874FFF0A3F0A3F0A3F0E4906EC8F081
:10138E00D20BC20CC20D908008E0F52630E405D2D7
:10139E00077410F0E52630E508D209908008742015
:1013AE00F0E52630E608D2089080087440F0E55F3C
:1013BE00C394034019908002E4F0908001F0908075
:1013CE0000F0E55F94064006E4F55F124DA29080B2
:1013DE00A0E07003124BB89080B8E07003124B3E41
:1013EE009080D0E07003124D46908000E070133074
:1013FE000710123EA3906B6BEFF0D39400400312D4
:10140E000026908002E07006908000E06005D20514
:10141E00021363C205E4F55F90693EE060030213B8
:10142E0063200B12906DB2E0600C7E1E7FA5123F02
:10143E00A7E4906DB2F0300912123848906B6BEF42
:10144E00F0D394004005E0FF125119200803021555
:10145E00D91236C1906B6BEFF07003021363906B71
:10146E00AFE054BF247F70030215421470030215BF
:10147E001A2402600302157B200B077E1E7FAC121E
:10148E003FA7200F030215D9906B87E07006906B73
:10149E008BE06067906EBCE0FF906B87E0B5072431
:1014AE00906EBDE0FE906B88E0B50618906EBEE0C3
:1014BE00FE906B89E0B5060C906EBFE0FE906B8AD5
:1014CE00E06E6037906B8BE06F60030215D9906E03
:1014DE00BDE0FF906B8CE06F60030215D9906EBE7D
:1014EE00E0FF906B8DE06F60030215D9906EBFE048
:1014FE00FF906B8EE06F60030215D9C203906DB141
:10150E007401F0120021755D010215D9906EC7E0CD
:10151E0060037401F0906EB4E0FF906BB1E06F6009
:10152E00030215D9906EB4E004F0E4F55D906DAF52
:10153E00F00215D93003030215D9906B7EE07003CB
:10154E00021363906B8F740AF012514DD203E4F5BF
:10155E005D906DAFF0906EC004F0E4906EB3F0A3AA
:10156E00F0200B677E1E7FBA123FA7805E906EC77B
:10157E00E060037401F0300352906BAFE020E74B54
:10158E00906BB1E0FF906EB3E0FE6F600D906EBB9E
:10159E00E07007EE146F70338013906EB3E004F0BA
:1015AE00906B6BE0FFD394044003124E8C90683A1C
:1015BE007482F0A37401F0906BB1E090683CF07E01
:1015CE00687F3A7D03124827021363200303021635
:1015DE00F1E55D7068124F71EF60237E6C7FAF9006
:1015EE006CB0E02404FD124827906EBBE0700990A9
:1015FE006B8FE0F55D021363E4F55D021363906E8D
:10160E00C0E0D3943C4036906EBBE07030906EC01C
:10161E0004F0125133E4906CAFF0A37412F0906E9C
:10162E00B4E0906CB1F0A374FDF090693F63A20139
:10163E00906CB363A2017F12123267809E12512802
:10164E008F26E526B4011590683A7483F0E4A3F072
:10165E007E687F3A7D02124827021363E526D394F3
:10166E0001401C90683A7483F0A37401F0E52624BF
:10167E00FEA3F07E687F3A7D03124827021363E5CE
:10168E005D64016003021363906DAFE004F0200B04
:10169E00077E1E7FC4123FA7906B8FE0C394C85085
:1016AE0004E02432F0906DAFE0C39405400DC20308
:1016BE00E4906DB1F01200210213637C6E7DBC903C
:1016CE006B83E0FAA3E0FB7F021249B87E6C7FAF1A
:1016DE00906CB0E02404FD124827906B8FE0F55D0E
:1016EE00021363E55D64016003021363906DB1E064
:1016FE0014604624FE60421470030217E424046052
:10170E0003021363E4F55F200F13906DB17404F0C0
:10171E00906DAFE05401F0755D010213639080028D
:10172E007410F0E4906DB1F0906DAF04F0755DFA49
:10173E00906EBC74FFF0021363906EBCE0700302F7
:10174E0017CE906CAF7480F0906CB17401F0E4A37E
:10175E00F0A304F0A37430F0A3747BF0E4F52674C8
:10176E00B62526F582E4346CF583747DF074B725C6
:10177E0026F582E4346CF583E4F0E5262407906CBC
:10178E00B0F07C6E7DBC906B83E0FAA3E0FB7F0231
:10179E001249B87E6C7FAFE5262409FD12482790CA
:1017AE006EBBE0601B12514DD203E4F55D906DAF40
:1017BE00F0906EC004F0E4906EB3F0A3F0021363E9
:1017CE00300F07E4906DB1F08006906DB17404F0A7
:1017DE00755DFA0213639080027410F0755D0590CA
:1017EE006DAFE06401FFF0906DB17401F0EF701910
:1017FE00906B8BE06013FCA3E0FDA3E0FEA3E0FF83
:10180E00906EBC122BA2021363906B87E0FCA3E0D8
:10181E00FDA3E0FEA3E0FF906EBC122BA2021363A9
:02182E0080FE3A
:011830002295
:10002600906BB0E0B444047F0180027F00906BAF18
:10003600E0B447047E0180027E00EE5F604A906B6A
:1000460078E0906BB1F0906B79E0906BB2F0906BCA
:100056007AE0906BB3F0906B7BE0906BB4F0906BB2
:100066007CE0906BB5F0906B7DE0906BB6F0906B9A
:10007600B07452F0906AE863A2019080A863A2016E
:100086007F061232670208F8906B6BE0C394085043
:1000960003020901906B78E0FF906BB1E06F60039B
:1000A600020901906B79E0FF906BB2E06F6003028A
:1000B6000901906B7AE0FF906BB3E06F6003020971
:1000C60001906B7BE0FF906BB4E06F600302090167
:1000D600906B7CE0FF906BB5E06F600302090190C6
:1000E6006B7DE0FF906BB6E06F6003020901906BD9
:1000F600B0E06444701A9080A8E0B4FF13906AE8F8
:1001060063A2019080A863A2017F06123267801065
:10011600906AECE09080ACF0906AEDE09080ADF0F3
:10012600906EC7E060037401F0906EC87464F0903E
:100136006BB07452F0906BAFE0646D600302029B8B
:100146007BFF7A1E79CF1223D57BFF7A1E79E99041
:100156006B78E0F52FA3E0F530A3E0F531A3E0F5E9
:1001660032A3E0F533A3E0F5341223D5752FFF75DE
:10017600301F7531467532FF75331F7534527BFF5C
:100186007A1F791F1223D57BFF7A1F795B1223D53D
:100196007BFF7A1F79C11223D57BFF7A1F79EE90F8
:1001A6006B7EE0F52FA3E0F530A3E0F531A3E0F593
:1001B600321223D57BFF7A207918906B87E0F52FD2
:1001C600A3E0F530A3E0F531A3E0F5321223D57BA9
:1001D600FF7A207946906B8BE0F52FA3E0F530A3EC
:1001E600E0F531A3E0F5321223D57BFF7A2079744E
:1001F600906B74E0F52FA3E0F530A3E0F531A3E0B2
:10020600F5321223D57BFF7A207997906B70E0F553
:100216002FA3E0F530A3E0F531A3E0F5321223D5A4
:100226007BFF7A2079B41223D57BFF7A2079DDA271
:100236000FE433F52F1223D57BFF7A21790D906ECB
:10024600BBE0F52F1223D57BFF7A217938906EC754
:10025600E0F52F1223D57BFF7A21796BA201E433D7
:10026600F52F1223D57BFF7A217997906EB5E0F5AD
:100276002FA3E0F530A3E0F531A3E0F532A3E0F5D6
:1002860033A3E0F5341223D5123C837BFF7A217920
:10029600E21223D522906BAFE0644C70737E217F0F
:1002A600E8FBFDFC123D9C906BB7E0F527A3E0F55B
:1002B60028E4F52AE527906BB9F0A3E528F07E221D
:1002C6007F237C6B7DB97B02123D9CE4F529852852
:1002D60082852783E0FF74B92529F582E4346BF51E
:1002E60083EFF00528E528700205270529E529B4DE
:1002F60010DC7E227F267C6B7DB97B10123D9C052F
:100306002AE52AC3941040AC7E227F29123FA722F9
:10031600906BAFE0646C7060F52B7E227F2BFBFD4B
:10032600FC123D9CE4F52AE4906BB9F0A3E52BF0B2
:100336007E227F237C6B7DB97B02123D9CE4F529EE
:10034600A82BE6FF74B92529F582E4346BF583EF13
:10035600F0052B0529E529B410E67E227F267C6B65
:100366007DB97B10123D9C052AE52AC3940840B747
:100376007E227F29123FA722906BAFE0644B70610B
:10038600F52974A12529F582E4346BF583E0603202
:1003960074A12529F582E4346BF583E0F4602374B7
:1003A600A12529F582E4346BF583E0FF74B725298E
:1003B600F582E4346BF583E0B507100529E529B429
:1003C60008C090693E7432F00208F8906BAF742151
:1003D600F0300B030208F87E227F66123FA7020860
:1003E600F8906BAFE0B4521A200B077E227F6E1294
:1003F6003FA7906BAF7472F07E6B7FAF7D0812479C
:10040600A022906BAFE064497045200B077E227FE7
:1004160079123FA7906BB7E0F527A3E0F528E4F53E
:1004260029852882852783E0FF74B92529F582E48A
:10043600346BF583EFF00528E528700205270529BA
:10044600E529B480DC7E6B7FAF7D8A1247A02290BF
:100456006BAFE064437046200B077E227F81123F1C
:10046600A7906BB7E0F527A3E0F528E4F5298528E2
:1004760082852783E493FF74B92529F582E4346BDA
:10048600F583EFF00528E528700205270529E529FB
:10049600B480DB7E6B7FAF7D8A1247A022906BAF64
:1004A600E0645A7053200B077E227F8A123FA79082
:1004B6006BB7E0F527A3E0F5287C6B7DB97B80AFB1
:1004C60028AE27124F3DE4F529852882852783E447
:1004D60093FF74B92529F582E4346BF583EFF005B3
:1004E60028E528700205270529E529B480DB7E6BFF
:1004F6007FAF7D8A1247A022906BAFE06444600311
:1005060002058F906BB7E0FF644470030208F8EFB2
:10051600B4310CC20B7E227F96123FA70208F890D8
:100526006BB7E0B4300CD20B7E227FA2123FA7023B
:1005360008F8906BB7E0B4320CD20C7E227FAF1273
:100546003FA70208F8906BB7E0B4330CC20C7E22CA
:100556007FBD123FA70208F8906BB7E0B4340CD207
:100566000D7E227FCC123FA70208F8906BB7E0B44D
:10057600350CC20D7E227FD9123FA70208F8906B78
:10058600B7E0FF12001E0208F890693EE0701320E3
:100596000B077E227FE7123FA7906BAF7421F00214
:1005A60008F890693E7432F0906BAFE0FFB45104E6
:1005B600C2AF80FEEF64577045200B077E227FF5A1
:1005C600123FA7906BB8E0906B6BF0E4F529906B47
:1005D6006BE0FFE529C39F40030208F874B925299B
:1005E600F582E4346BF583E0FF906BB7E0252924B0
:1005F600E7F582E43469F583EFF0052980D0906B46
:10060600AFE0645360030206B2200B077E237F002F
:10061600123FA7906B78E0FF9069F0E06F703C9016
:100626006B79E0FF9069F1E06F7030906B7AE0FFD4
:100636009069F2E0B50724906B7BE0FF9069F3E0E8
:10064600B50718906B7CE0FF9069F4E0B5070C9055
:100656006B7DE0FF9069F5E06F6016906BAF7421DB
:10066600F0300B030208F87E237F0F123FA7020823
:10067600F8E4F529E4F560AF29FE74E72529F5824B
:10068600E43469F583E0FD1250210529E529C39478
:10069600FE40E1C2AFE4907FF0F0A3F0907FFD74DE
:1006A600AAF0A374FFF0A37455F080FE906BAFE040
:1006B600644F705A906BB7E0F527A3E0F528E5285C
:1006C6004527700A200B077E237F18123FA7200BB1
:1006D600077E237F1F123FA7E4F52974B92529F564
:1006E60082E4346BF583E0852882852783F005282C
:1006F600E528700205270529E529B480DE906EC637
:10070600E02480F0906EC5E03400F00208F8906BAB
:10071600AFE064457074906BB7E0FEA3E0FF907F96
:10072600F0EEF0A3EFF0D39400EE94044038907FFF
:10073600F0E0FEA3E0FF906EC5E0FCA3E0FD9FECB9
:100746009E4023E42FFFEE3401FED3ED9FEC9E5036
:1007560015C2AF907FFD74AAF0A374FFF0A3745581
:10076600F0E4F5A780FE7E237F21123FA77BFF7A68
:10077600237929907FF0E0F52FA3E0F530906EC540
:10078600E0F531A3E0F5321223D5906BAFE0646556
:100796006003020901906BB7E0FFA3E0907FF0CF02
:1007A600F0A3EFF0E4F527F528D3907FF1E0952844
:1007B600907FF0E095274020E4F5602528FFE527A7
:1007C6003401FE852882852783E0FD125021052805
:1007D600E5287002052780D17E237F341248AEEFCC
:1007E6004E6020120003906B7EEFF0120003906BB8
:1007F6007FEFF0120003906B80EFF0120003906B16
:1008060081EFF07E237F3A1248AEEF4E6020120051
:1008160003906B87EFF0120003906B88EFF01200E5
:1008260003906B89EFF0120003906B8AEFF07E2342
:100836007F401248AEEF4E6020120003906B8BEFA4
:10084600F0120003906B8CEFF0120003906B8DEFAB
:10085600F0120003906B8EEFF07E237F461248AEB7
:10086600EF4E6020120003906B74EFF012000390BD
:100876006B75EFF0120003906B76EFF012000390A9
:100886006B77EFF07E237F4C1248AEEF4E6020125E
:100896000003906B70EFF0120003906B71EFF01293
:1008A6000003906B72EFF0120003906B73EFF0E4AD
:1008B600F529E4F560E5292401FFE433FE7470258B
:1008C60029F582E4346BF583E0FD1250210529E514
:1008D60029C3944340DCC2AFE4907FF0F0A3F090CC
:1008E6007FFD74AAF0A374FFF0A37455F0E4F5A796
:0B08F60080FE7E6B7FAF7D081247A0E4
:0109010022D3
:104F0500AE07EEC39430400BEED394395005EE2432
:104F1500D0FF22EEC39461400BEED394665005EEAC
:104F250024A9FF22EEC39441400BEED394465005CD
:084F3500EE24C9FF22AF0622A1
:1050C700906AE7E004F07006906AE6E004F0906A00
:0A50D700E6E0FEA3E0FF12508D2278
:100003001250C7124F05EFC454F0FEC0061250C77A
:08001300124F05D0E02FFF227F
:104CE900E4907021F01250C7907022EFF0C3943015
:104CF9004018E0FFD394395011907021E0243FF51A
:104D090082E43469F583EFF08011907021E0243F4B
:104D1900F582E43469F583E4F0800C907021E004B5
:104D2900F0E0D3940840BE75320075330075340045
:0C4D3900E4F5357B017A69793F12351DE5
:014D4500224B
:0448AE008E2C8F2D90
:1048B200906AE6E4F0A374FFF01250C7EF606EF462
:1048C200606B852D82852C83E493B507EC752E01F0
:1048D200E52D252EF582E4352CF583E493602590B1
:1048E2006AE7E0252EFF906AE6E03400FE12508D62
:1048F200E52D252EF582E4352CF583E493B50704E6
:10490200052E80CCE52D252EF582E4352CF583E4A9
:104912009370A6E52E24FFFFE434FFFE906AE7E0E1
:104922002FF0906AE6E03EF07E007F0122E4FEFF77
:014932002262
:104320007E237F521248AEEF4E70037F01227E2320
:104330007F551248AEEF4E600C1250C7EF24D024C8
:10434000FF920F8002D20F7E237F5B1248AEEF4EAA
:10435000600C1250C7EF24D0906EBBF08005E49043
:104360006EBBF07E237F611248AEEF4E600C1250A0
:10437000C7EF24D0906EC7F08005E4906EC7F07E42
:10438000237F671248AEEF4E600C1250C7EF24D067
:1043900024FF92018002C201906B7863A201906EAB
:1043A000B563A2017F0612326730013B7E237F6D29
:1043B0001248AEEF4E6030120003906EB5EFF0126F
:1043C0000003906EB6EFF0120003906EB7EFF0129C
:1043D0000003906EB8EFF0120003906EB9EFF01288
:0A43E0000003906EBAEFF07F002298
:104DFC00906DB0E0C3947C40027F0A906DB0E0FEF1
:104E0C0004F074EE2EF582E4346AF583EFF0BF0AF9
:104E1C0027906DB0E0FF04F074EE2FF582E4346A55
:104E2C00F583E4F0906DB0E0FF124933906DB074EF
:094E3C0008F0906AEFE004F02296
:104DA2009080007480F0906B7063A201F583F582AD
:104DB20063A2017F08123267906B7863A201908030
:104DC2008863A2017F0A1232679080927407F0A36F
:104DD20074D0F0A37406F0906B82E0FF9080B1F083
:104DE2009080E1EFF09080957455F0A3F0908000F0
:0A4DF2007401F090800974F0F022C3
:104BB800908009E04410F09080A0E070609080A19F
:104BC8007482F09080A874FFF0A3F0A3F0A3F07FA4
:104BD800039080AEEFF0A374CBF09080007402F0E5
:104BE800907015122BAE00000000907015E09080B8
:104BF80040F0907016E0908041F0907017E090803F
:104C080042F0907018E0908043F0A3E4F0A3F0A382
:0D4C1800F0A3F0908018F0A3F0A3F0A3F03B
:014C2500226C
:104D4600908009E04440F09080D17482F07F039017
:104D560080DEEFF0A374CCF09080027402F09070C5
:104D660019122BAE00000000907019E0908058F0E8
:104D760090701AE0908059F090701BE090805AF085
:104D860090701CE090805BF0A3E4F0A3F0A3F0A386
:0B4D9600F0908030F0A3F0A3F0A3F039
:014DA10022EF
:104B3E00908009E04420F09080B8E0706C9080B9CD
:104B4E007482F07F039080C6EFF07FCDA3EFF07FED
:104B5E00039080C4EFF0A374CDF09080C074FFF08A
:104B6E00A3F0A3F0A3F09080017402F090701D12D8
:104B7E002BAE0000000090701DE090804CF0907005
:104B8E001EE090804DF090701FE090804EF090707F
:104B9E0020E090804FF0A3E4F0A3F0A3F0A3F090F8
:094BAE008024F0A3F0A3F0A3F0B1
:014BB70022DB
:1049B8008C278D28A907EAFDE975F018A424ACFF17
:1049C800E5F034808F82F583EDF0EBFDE975F018A2
:1049D800A4FFAEF024ACFBEE34808B82F583A3ED0C
:1049E800F08528828C83E0FDEF24A8FFEE3480FE5A
:1049F8008F82F583EDF08528828C83A3E08F828EE9
:104A080083A3F0852882852783A3A3E0FDE975F0B9
:104A180018A424A8FFE5F03480FE8F82F583A3A3B1
:104A2800EDF08528828C83A3A3A3E08F828E83A3D5
:044A3800A3A3F02222
:0647A0008D2CAB07AA06F8
:1047A600908000E030E507906DB27401F0229070C1
:1047B60015E0FCA3E0FDA3E0FEA3E0F5308E2F8D0F
:1047C6002E8C2DAE02AF038E838F8263A201E52F5E
:1047D600540744C0F58385308263A201AF2C1232A0
:1047E600D9E4FCFDFEE530252CF530EE352FF52F0E
:1047F600ED352EF52EEC352DF52D908040E52DF07E
:10480600A3E52EF0A3E52FF0A3E530F09080007429
:1048160020F0AF30AE2FAD2EAC2D907015122BA21E
:01482600226F
:064827008D27AB07AA0675
:10482D00908002E030E507906DB27403F022907035
:10483D0019E0FCA3E0FDA3E0FEA3E0F52B8E2A8D8D
:10484D00298C28AE02AF038E838F8263A201E52AE5
:10485D00540744D0F583852B8263A201AF27123212
:10486D00D9E4FCFDFEE52B2527F52BEE352AF52A9F
:10487D00ED3529F529EC3528F528908058E528F0F7
:10488D00A3E529F0A3E52AF0A3E52BF090800274AF
:10489D0020F0AF2BAE2AAD29AC28907019122BA2A7
:0148AD0022E8
:02449C008F2867
:10449E00908001E030E509906DB27402F07F002249
:1044AE0090701DE0FCA3E0FDA3E0FEA3E0F52C8ED2
:1044BE002B8D2A8C29906EB563A201E52B540744EF
:1044CE00C8F583852C8263A2017F061232EFE52C9C
:1044DE002406F52CE4352BF52BE4352AF52AE435A4
:1044EE0029F529906DB363A201E52B540744C8F555
:1044FE0083852C8263A201AF281232EFE4FCFDFE0D
:10450E00E52C2528F52CEE352BF52BED352AF52A45
:10451E00EC3529F52990804CE529F0A3E52AF0A386
:10452E00E52BF0A3E52CF09080017420F0AF2CAEBB
:0D453E002BAD2AAC2990701D122BA2AF28C6
:01454B00224D
:103EA3009081E0E0F5270527052705270527052746
:103EB30005270527052705270527908010E0F52A04
:103EC300A3E0F52BA3E0F52CA3E0F52D9081E1E031
:103ED300F52705270527052705270527052705278F
:103EE300052705270527908014E0F52EA3E0F52F7D
:103EF300A3E0F530A3E0F531E530B52C08E531B5A5
:103F03002D037F0022E4F527E530540744E0F583D1
:103F130085318263A201906BAF63A2017F081233E4
:103F23001F906BB163A201906AE863A2017F06123E
:103F33003267906BAFE0F528A3E0F529E4F527900D
:103F43006BAFE0702AA3E024F8F527E5305407446B
:103F5300E0F58385318274082582F582E43583F5A3
:103F63008363A201906BAF63A201AF2712331FAE2D
:103F730028E4FCFDE5312529F531E5303EF530ED4A
:103F8300352FF52FEC352EF52E908014E52EF0A36A
:103F9300E52FF0A3E530F0A3E531F0908000744005
:033FA300F0AF2755
:013FA60022F8
:1036C1009081E6E0F527052705270527052705272A
:1036D10005270527052705270527908028E0F52AD6
:1036E100A3E0F52BA3E0F52CA3E0F52D9081E7E015
:1036F100F527052705270527052705270527052779
:1037010005270527052790802CE0F52EA3E0F52F4E
:10371100A3E0F530A3E0F531E4F527E530B52C0A57
:10372100E531B52D05C20802382DE530540744F0C6
:10373100F58385318263A201906BAF63A2017F089B
:1037410012331F906BAFE0F528A3E0F529E5294579
:103751002870099080027410F07F0022906EBCE006
:10376100FFF46030906BB1E06F60030237F4906E4C
:10377100BDE0FF906BB2E06F7079906EBEE0FF909C
:103781006BB3E06F706D906EBFE0FF906BB4E06F54
:103791006031805F906BB1E0906EBCF0906BB2E0F5
:1037A100906EBDF0906BB3E0906EBEF0906BB4E0A4
:1037B100906EBFF0906BB5E0FFA3E0906B83CFF00C
:1037C100A3EFF0906BAFE0702AA3E024F8F527E5B2
:1037D10030540744F0F58385318274082582F582DF
:1037E100E43583F58363A201906BAF63A201AF2738
:1037F10012331FAE28E4FCFDE5312529F531E53012
:103801003EF530ED352FF52FEC352EF52EAF2DAEE3
:103811002CAD2BAC2AAB31AA30A92FA82ED3122B59
:103821009140099080027410F07F002290802CE575
:103831002EF0A3E52FF0A3E530F0A3E531F0908061
:06384100027440F0AF2705
:01384700225E
:103848009081E3E0F52705270527052705270527A4
:103858000527052705270527052790801CE0F52A59
:10386800A3E0F52BA3E0F52CA3E0F52D9081E4E08F
:10387800F5270527052705270527052705270527F0
:10388800052705270527908020E0F52EA3E0F52FD2
:10389800A3E0F530A3E0F531E4F527E530B52C0ACF
:1038A800E531B52D05C20902399EE530540744E8D3
:1038B800F58385318263A20190683E63A2017F0E81
:1038C80012333590683EE0F528A3E0F52990684664
:1038D800E0FFF4604A906EB5E0FEEF6E7079A3E009
:1038E800FF906847E06F706F906EB7E0FF90684890
:1038F800E06F7063906EB8E0FF906849E06F7057B2
:10390800906EB9E0FF90684AE06F704B906EBAE035
:10391800FF90684BE06F703FE490684DF08008902E
:10392800684D74FFF0D2D990683EE0702AA3E02475
:10393800F2F527E530540744E8F583853182740EA3
:103948002582F582E43583F58363A20190683E639E
:10395800A201AF27123335AE28E4FCFDE531252955
:10396800F531E5303EF530ED352FF52FEC352EF5F8
:103978002EAF2DAE2CAD2BAC2AAB31AA30A92FA877
:103988002ED3122B915006E5294528700990800105
:103998007410F07F0022908020E52EF0A3E52FF030
:1039A800A3E530F0A3E531F09080017440F0AF2733
:0139B80022EC
:043FA7008E2D8F2E9E
:103FAB00908000E030E507906DB27401F0229070C4
:103FBB0015E0FCA3E0FDA3E0FEA3E0F5348E338D0A
:103FCB00328C31E534FFE5335407FEE42FF530EE48
:103FDB0034C0F52F853082F5837423F00530E5303E
:103FEB007002052F532FC7F582852F83740AF005B6
:103FFB0030E5307002052F532FC7906B7863A20109
:10400B00852F8385308263A2017F061232D9740615
:10401B002530F530E4352FF52F852D83852E8263E2
:10402B00A201852F8385308263A2011232BDE4FC8D
:10403B00FDFE907015E0F8A3E0F9A3E0FAA3E02FE2
:10404B00FFEE3AFEED39FDEC38FCEF2408FFE43EC1
:10405B00FEE43DFDE43CFC907015122BA290701514
:10406B00E0908040F0907016E0908041F0907017D7
:10407B00E0908042F0907018E0908043F0908000C8
:03408B007420F0AE
:01408E00220F
:0A3D9C008E2C8F2D8C2E8D2F8B3076
:103DA600908000E030E507906DB27401F0229070CB
:103DB60015E0FCA3E0FDA3E0FEA3E0F5368E358D0D
:103DC600348C33E536FFE5355407FEE42FF532EE45
:103DD60034C0F531853282F5837423F00532E5323D
:103DE600700205315331C7F582853183740AF005B7
:103DF60032E532700205315331C7906B7863A20108
:103E060085318385328263A2017F061232D9740618
:103E16002532F532E43531F531852C83852D8263E3
:103E2600A20185318385328263A2011232BD8F37AA
:103E3600EF2532F532E43531F531E5306017852E60
:103E460083852F8263A20185318385328263A20135
:103E5600AF301232D9E53724082530F530FFE4FCBF
:103E6600FDFEE5362FF536EE3535F535ED3534F50F
:103E760034EC3533F533908040E533F0A3E534F088
:103E8600A3E535F0A3E536F09080007420F0AF3658
:0C3E9600AE35AD34AC33907015122BA289
:013EA20022FD
:064170008E2D8F2E8D2F15
:10417600908000E030E507906DB27401F0229070F7
:1041860015E0FCA3E0FDA3E0FEA3E0F5358E348D3B
:10419600338C32E535FFE5345407FEE42FF531EE76
:1041A60034C0F530853182F5837423F00531E5316D
:1041B600700205305330C7F582853083EBF0053148
:1041C600E531700205305330C7906B7863A20185E4
:1041D600308385318263A2017F061232D9740625A7
:1041E60031F531E43530F530852D83852E8263A295
:1041F6000185308385318263A201AF2F1232D974D3
:1042060008252FF52FFFE4FCFDFEE5352FF535EEED
:104216003534F534ED3533F533EC3532F5329080FF
:1042260040E532F0A3E533F0A3E534F0A3E535F03D
:104236009080007420F0AF35AE34AD33AC32907060
:0442460015122BA280
:01424A002251
:024933008F40B3
:10493500908000E030E507906DB27401F022907030
:1049450015E0FCA3E0FDA3E0FEA3E0F5448E438D56
:10495500428C41E544FFE5435407FEE42FFFEE3466
:10496500C0906AEE63A201F5838F8263A201AF4016
:104975001232D9E4FCFDFEE5442540F544EE35430D
:10498500F543ED3542F542EC3541F541908040E582
:1049950041F0A3E542F0A3E543F0A3E544F09080A0
:1049A500007420F0AF44AE43AD42AC419070151297
:0249B5002BA233
:0149B70022DD
:06408F008E2A8F2BAB0509
:10409500908000E030E507906DB27401F0229070D9
:1040A50015E0FCA3E0FDA3E0FEA3E0F5318E308D25
:1040B5002F8C2EE531FFE5305407FEE42FF52DEE6C
:1040C50034C0F52C852D82F5837423F0052DE52D5F
:1040D5007002052C532CC7F582852C83EBF0052D3A
:1040E500E52D7002052C906B7863A201852C8385E4
:1040F5002D8263A2017F061232D97406252DF52D76
:10410500E4352CF52C532CC7E52A852D82852C8387
:10411500F0052DE52D7002052C532CC7F582852C55
:1041250083E52BF0052DE52D7002052C532CC7E5F5
:1041350031240AF531E43530F530E4352FF52FE437
:10414500352EF52E908040E52EF0A3E52FF0A3E562
:1041550030F0A3E531F09080007420F0AF31AE303F
:0A416500AD2FAC2E907015122BA2A6
:01416F00222D
:10508D00A2AF9220C2AF438E2075D2028F828E8343
:0C509D00E0FFE4F5D2538EDFA22092AFBA
:0150A90022E4
:10502100E5D220E0FBA2AF9220C2AF43D2028F8231
:105031008E83EDF075D25063D250A22092AFE5D2AB
:0350410020E0FB71
:015044002249
:104AC000E4FDED2401FFE433FE12508D74702DF5EA
:104AD00082E4346BF583EFF00DBD3FE6E4FDED2499
:104AE0007FFFE433FE12508D74672DF582E4346944
:104AF000F583EFF074672DF582E43469F583E07097
:104B00001B74672DF582E43469F5837420F07468B2
:104B10002DF582E43469F583E4F080040DBD80BE98
:104B2000E49069E6F0FDEDFF7E0012508D74E72DF4
:0D4B3000F582E43469F583EFF00DBDFEE978
:014B3D002255
:024F3D008B2CBB
:104F3F00A2AF9220C2AF85A22D53A2FE8E838F8285
:104F4F0005A28C838D827409123363E52C53A2FE64
:104F5F0043A22012336553A2DF852DA2A22092AF68
:014F6F00FF42
:014F7000221E
:1050AA00A2AF9220C2AF8C838D82EF12336343A2E8
:0C50BA002012336553A2DFA22092AFFF4A
:0150C60022C7
:025045008F27B3
:10504700A2AF9220C2AFE4F5838D82740612336358
:10505700E52743A22012336553A2DFA22092AF7F38
:015067000147
:015068002225
:025069008F278F
:10506B00A2AF9220C2AFE4F5838D82740A12336330
:10507B00E52743A22012336553A2DFA22092AF7F14
:01508B000123
:01508C002201
:10318C00A907E7FFA805EF93C3966008403B74FCC2
:10319C002FFF80F00F08EF93C3966008402B74FB51
:1031AC002FFF80E00F08EF93C3966008401B74FA62
:1031BC002FFF80D00F08EF93D3966008400B74F963
:1031CC002FFF80C01F1F1F1F1FEF54FEF80303F7B4
:1031DC00E893FC08E893FD08E893FE08E893FF22C7
:1031EC0009E993C39D6008402974FB29F980F10912
:1031FC00E993C39E6008401A74FA29F980E209E940
:10320C0093D39F6008400B74F929F980D3191919CD
:10321C001919E9C313C313FF22740093F8ECC39874
:10322C004024701F740193F8EDC398401970147406
:0E323C000293F8EEC398400E7009740393F8E5
:10324A00EFC39840037F00227F0122EDF8E6F008E1
:10325A00A3DFFA22EDF8E0F608A3DFFA22E0A3637F
:10326A00A201F0A363A201DFF475A2002263A20106
:10327A00F0A363A20122E0A363A201F0A363A20167
:10328A00E0A363A201F0A363A201E463A201F0A395
:10329A0063A201DFE175A20022E0A363A2016DFE31
:1032AA00936CFDEE058393FC158363A201DFEA7537
:1032BA00A200227F00E493A363A201F00F600CA393
:1032CA00E583C2E3F58363A20180EA75A20022E0E6
:1032DA00A363A201F0A3E583C2E3F58363A201DF3E
:1032EA00EE75A20022E0A363A201F0A3E583C2E483
:1032FA00D2E3F58363A201DFEC75A20022E0A363A7
:10330A00A201F0A3E58344F8C2E5F58363A201DFD5
:10331A00EC75A20022E583C2E3F583E0A363A20170
:10332A00F0A363A201DFEE75A20022E583C2E4D214
:0A333A00E3F583E0A363A201F0A312
:1033440063A201DFEC75A20022E58344F8F583E073
:10335400A363A201F0A363A201DFEE75A20022F928
:1033640022C002C004C00612FFF0D006D004D0026E
:013374002236
:10454C004572724C656E210A000A496E49503A0058
:10455C00205544502054696D654750530A00200A79
:10456C00495054696D653A2000200A444154414732
:10457C0052414D3A20002049676E6F72650A200047
:10458C002043414E2054696D654750530A00205416
:10459C007261737353656E644552520A000ACEF809
:1045AC00C4EBE8EDFB43414E210A000A457272410F
:1045BC00647243414E3A00205265496E697420433F
:1045CC00414E0A002043414E283029203E20544FB2
:1045DC00210A0020545520300A0020545520310A5D
:0145EC0000CE
:03001E00E4FF22DA
:104FD200C2A9438902758C48758A4875D90475DB64
:104FE2004875DC4875DD4875DE48E4F5E9F5F9D227
:084FF200D9C2DAD28CD2DE2212
:104FA400C2D9906EDDE07013E5E92419F5EB30D732
:104FB40006E5F904F5FB2285F9FB22E5E924C8F5A9
:0E4FC400EB30D706E5F904F5FB2285F9FB2258
:104E4500C2D9906EDDE0702C302D16E5E92432F5DF
:104E5500EB30D707E5F904F5FB800385F9FBC22D97
:104E650022E5E92405F5EB30D706E5F904F5FB2243
:104E750085F9FB22E5E92432F5EB30D706E5F9049F
:074E8500F5FB2285F9FB2279
:104FFA00124FD2906EDDE0C394645006124A3C12FE
:10500A004FA4125153D22CE4F556906FF5F0F545A2
:07501A00F55AC22DF55822E2
:104E8C00EF24FCF545D3940D4010200B077E457F95
:104E9C004C123FA7E4F545D22A22906BB363A201D2
:104EAC00906FE563A201AF45123267C22A200B0D49
:0E4EBC007E457F557C6B7DB3AB45123D9C223D
:0F511900D3EF6480948D5006E55A70028F5A22AE
:1026CF0020D9030227D3202C030227D3E55A6067B2
:1026DF0090683E540FFF7D4712325EE547640170EC
:1026EF003A90684DE0B4FF0ED22E200B127E457F3C
:1026FF005C123FA78009302E06E4F55A0227D31249
:10270F004FA4124C26200B0D7E457F6A7C687D3EC0
:10271F00AB5A123D9CE4F55A0227D3124FA4124C28
:10272F0026200B0D7E457F757C687D3EAB5A123D92
:10273F009CE4F55A0227D3E5456055906FE9E024F4
:10274F0005F527D3940D4007E4F545D22A807590FF
:10275F006FE5E527540FFF7D4712325EE54730E7FF
:10276F0002D22DE5476401701A302E17E54AB401E5
:10277F0012200B127E457F827C687D3EAB5A123D44
:10278F009C8003124C26124FA4E4F545D22A8034C4
:10279F00E557601E906EC9540FFF7D4712325EE5FC
:1027AF0047B40103202E03124C26124FA4E4F55711
:1027BF00801220110C906EDDE0C39464500312421E
:1027CF004B124FA4123B288F27EF70030228FCE413
:1027DF00F558E54730E70AE54AB41905D2D902287A
:1027EF00FC124E45E547B4010CD22E200B077E4557
:1027FF007F8C123FA7E559C394C8501B3003187440
:10280F00DE2559F582E4346EF583E5272559F55910
:10281F007D47AF27123255300121E54720E71C9045
:10282F006DB37D47AF27123255AF2712449CEF701F
:10283F000A200B077E457F9A123FA7E54754816018
:10284F00030228FCE527D3940D4010300B03022818
:10285F00FC7E457FA9123FA70228FCE549D39407C8
:10286F00401F300B030228FC90693F7D47AF2712B2
:10287F0032557E457FB77C697D3FAB27123D9C80EB
:10288F006CE51330E662907010E0FF904CB793FE4A
:10289F00547F65477052EFA3936549704B9070104A
:1028AF00E0C313FF24F7F582E4346FF583E070384B
:1028BF0053133F907010E0FD74872513F582E434B5
:1028CF0061F583EEF0ED904CB893FE74882513F507
:1028DF0082E43461F583EEF074F72FF582E4346F00
:1028EF00F5837401F0431340AF27122CE0300E1A1A
:1028FF00300015906EDDE0C39464500C0558E55818
:10290F0094F04004C2AF80FEC20E200203022A14CC
:10291F00E5566031D39401400415568028906FF529
:10292F00E004F0E0D39403400D200B077E457FC3F6
:10293F00123FA7124FFA200B077E457FD0123FA7F9
:10294F00E4F556D22CE5576003022A12302B3F9044
:10295F006EC904F0A37408F0A37480F0A37401F09F
:10296F00A37406F0906FE0E0906ECEF0906FE1E010
:10297F00906ECFF0906FE2E0906ED0F0906FE3E04A
:10298F00906ED1F0E4A3F0A3F075570BC22B302952
:10299F0072906FDEE07035E5577031906EC97442FA
:1029AF00F0A37408F0906FDFE0906ECBF0906FE4BF
:1029BF00E0906ECCF0A37401F0755706200B077EE4
:1029CF00457FDF123FA7906FDEE004F0906FDEE0EF
:1029DF006402702FE557702B906EC97402F0A374C8
:1029EF0008F0906FDFE0906ECBF0A3F0A37401F0CE
:1029FF00755706200B077E457FE6123FA7906FDEC7
:0A2A0F00E004F0C202120902C20046
:012A1900229A
:104F7100E559602CE4906CAFF0A3E559F0906EB464
:104F8100E0906CB1F0A37419F0906EDE63A2019011
:104F91006CB363A201AF59123267E4F5597F012264
:034FA1007F00226C
:0B512800302A05C22A7F01227F0022EE
:0100210022BC
:06514D00E4F559F54522CE
:0A513300E490693FF0A3F0A3F0221E
:104C88002043616E457247495400200A00457272FC
:104C98004C656E43616E21000A002043616E4572C7
:104CA80072434821000A205265714572722100C47E
:104CB80000C401C402C403C404C405C406C407C8AC
:104CC80000C801C802C803C804C805C806C807C286
:104CD80000C201C202C203C204C205C206C2070062
:014CE80000CB
:103B2800E59B541F6020200B1A7E4C7F88123FA70C
:103B3800E59B541FFF7E007D0312408F7E4C7F92D1
:103B4800123FA7E4F59BE5BA30E010E4F5B375B190
:103B580080F5B2D22CF556906FF5F0E5CFF47003EE
:103B6800023C80752901E4F528E5CFF45529700356
:103B7800023C6EE528C454F0F5B1E5B2547F6420E8
:103B88006003023C3FE5B3540FF54B85BC47E5BDE8
:103B9800541FFF131313541FFFE5BD54E044184F7F
:103BA800F548E5BDC43354E0FFE5BE131313541FB5
:103BB8004FF549E5BEC43354E0FFE5BF1313135472
:103BC8001F4FF54A85A34C85A34D85A34E85A34F6A
:103BD80085A35085A35185A35285A353E4F5B2204C
:103BE800110FE547547EB5470843BDF875B35080BB
:103BF8000375B3D0E54B700AE547547EB547037F9C
:103C08000022301108E54730E7037F0022E54BD357
:103C18009408401D200B177E4C7F95123FA7AF4B91
:103C28007E007D0312408F7E4C7FA0123FA77F004D
:103C380022E54B2405FF22E5B2549F6023200B2088
:103C48007E4C7FA2123FA7AFB27E007D0312408F49
:103C5800AFB37E007D0312408F7E4C7FA0123FA73A
:103C6800E4F5B275B3D0E52925E0F5290528E5285E
:0A3C7800C394085003023B717F0063
:013C8200221F
:104C2600906EDDE0C39464505675B180E4F5B3F53B
:104C3600B28547BCE549C4135407FFE54854E04F25
:104C4600F5BDE54933333354F8FFE54AC413540739
:104C56004FF5BEE54A33333354F8F5BF854CA3858B
:104C66004DA3854EA3854FA38550A38551A3855299
:104C7600A38553A3E54B540F2450F5B375560AC2CA
:024C86002C22DE
:10424B0075B190E5B220E613200B107E4C7FAD12BA
:10425B003FA7AFB27E007D0312408FE4F5B3F5B2FA
:10426B00E51330E615E4F513907010E02402F0E04E
:10427B00904CB7937004907010F074872513F582EF
:10428B00E43461F583E0702D907010E0FFC31324CC
:10429B00F7F582E4346FF583E070054313808015E6
:1042AB00E4F513907010E02402F0E0904CB793709B
:1042BB0004907010F0E51330E721907010E0FF9040
:1042CB004CB793F5BCE4F5BDEFA393FF33333354F5
:1042DB00F8F5BE75BF78431340803674872513F508
:1042EB0082E43461F583E0F5BC75BD8074882513D9
:1042FB00F582E43461F583E0FF33333354F8F5BED4
:10430B0075BF7805130513E513C394324003E4F529
:05431B001375B35022F0
:09513D00EF6003C29622D2962213
:104A3C0043AB01C2E8C2EAE4FFEFC454F0F5B1C3E2
:104A4C00EF64809488500575B3D08003E4F5B3E42B
:104A5C00F5B2F5BCF5BDF5BEF5BFF5C4F5C5F5C6AB
:104A6C00F5C7F5A3F5A3F5A3F5A3F5A3F5A3F5A356
:104A7C00F5A30FBF0EC3906EDDE0FE25E0F5B47517
:104A8C00B50C75B66C75A11275AB0275C13E75C3CC
:104A9C00FF75C203E4907010F0751380FF7F1990BE
:104AAC006FF7E4F0A3DFFCE4FF7F32906187E4F062
:034ABC00A3DFFC79
:014ABF0022D4
:101831005452414E5A004D415842005254530044B3
:10184100454C4159004D4F4445004B500054550003
:1018510043414E004B565400415400444952004309
:10186100414E4D4F4E00475254494D450054495445
:1018710053005453494E5600003E2A2C312CCFE0E0
:10188100F0E0ECE5F2F0FB20F3EFF0E0E2EBFFFE3D
:10189100F9E5E3EE20EAEEEDF2F0EEEBEBE5F0E058
:1018A10020CACF20C8F1E5F2FC0A003E4C2C6B3077
:1018B100312C25732C43EAEEF0EEF1F2FC20EDE041
:1018C10020F8E8EDE52043414E2C30202D20353025
:1018D10030EAE1283530EC292C31202D203530EA51
:1018E100E128353030EC290A0030202D2035303008
:1018F100EAE1283530EC290031202D203530EAE1AC
:1019010028353030EC29003E532C6B30322C2562C7
:10191100752CCCE0EAF12E20E0E4F0E5F120E1EBDA
:10192100EEEAE020D2D128302D38290A003E532C8E
:101931006B30332C2562752CCCE0EAF12E20E0E4EB
:10194100F0E5F120E1EBEEEAE020D2C8D228302D1B
:1019510038290A003E532C6B30342C2562752CCC6F
:10196100E0EAF12E20E0E4F0E5F120E1EBEEEAE03F
:1019710020D2D328302D38290A003E422C63303141
:101981002C2562752CC2F2EEF0E8F7EDFBE920EAB6
:10199100EEEDF2F0EEEBEBE5F020EDE020F8E8ED16
:1019A100E50A003E2A2C312CCFE0F0E0ECE5F2F024
:1019B100FB20EFF0EEF2EEEAEEEBE020C3F0E0ED1B
:1019C100E8F220EFEE20EFEEF0F2F3205253323343
:1019D100320A003E432C61636B2C25732CCFEEF051
:1019E100FFE4EEEA20C0D4C10A00312DD2D1283063
:1019F1002B312920322DD2C8D228302920332DD2A3
:101A0100D320342DD2C8D228312920352DD2D12846
:101A1100322B332920382DD2C8C8003E4C2C6B30D4
:101A2100352C256C752CD1EAEEF0EEF1F2FC20EEAE
:101A3100E1ECE5EDE020EDE020EFEEF0F2F32C310A
:101A410030302C3230302C3330302C3630302C3199
:101A51003230302C323430302C343830302C39366E
:101A610030302C31393230302C33383430302C3561
:101A7100373630302C3131353230300A003E532C7C
:101A81006B30362C2562752CCDEEECE5F020CACFFB
:101A9100200A003E422C6730312C2562752CCCE0A7
:101AA100E3E8F1F2F0E0EBFC0A003E422C67303251
:101AB1002C2562752CC8EDE2E5F0F2E8F0EEE2E0EB
:101AC100F2FC20E7EDE0F7E5EDE8FF20D2D10A00D6
:101AD1003E422C6730332C2562752CC7E0EFF0E0D5
:101AE100F8E8E2E0F2FC20E2F0E5ECFF20F1E5F0BD
:101AF100E2E5F0E00A003E422C6730342C256275A5
:101B01002CC2FBF1F2E0E2EBFFF2FC205254532035
:101B1100EFF0E820EFE5F0E5E4E0F7E50A003E53F9
:101B21002C6730352C2562752CC7E0E4E5F0E6EA38
:101B3100E020EFE5F0E5E4E0F7E820EFEEF1EBE59A
:101B41002052545320282A3130ECF1290A003C213B
:101B5100003C6B30313D003C6B30323D003C6B3022
:101B6100333D003C6B30343D003C6330313D003C43
:101B71006B30353D003C6B30363D003C6730313DCC
:101B8100003C6730323D003C6730333D003C6730FC
:101B9100343D003C6730353D000ACFE5F0E5E4E037
:101BA100F7E03A2000544949204379636C650A0003
:101BB1005453204379636C650A0054530A00544915
:101BC100540A005455204F4B0A0054552044696172
:101BD100670A005455205265710A0020545520545B
:101BE100696D654F5554210A000ACFF0E8E5EC3ADA
:101BF10020000A4352432045525221000AD7F3E6FE
:101C0100EEE920EDEEECE5F020CACF21000A5265A5
:101C11007154533120000A52657154533520000A22
:101C210052657154495420000ACFF0E8EDFFF2E00B
:101C310020EAEEECE0EDE4E020D2D320002020D237
:101C4100D320E7E0EDFFF2EE210A000ACDE520EF17
:101C5100EEEDFFEB20F2E8EF20EFE0EAE5F2E02124
:101C61000A0000112332465765748C9DAFBECADB52
:101C7100E9F810013322564775649C8DBFAEDACB6B
:101C8100F9E82130021367764455ADBC8E9FEBFA1B
:101C9100C8D93120120377665445BDAC9E8FFBEA4B
:101CA100D8C94253617004152736CEDFEDFC8899FF
:101CB100ABBA5243716014053726DECFFDEC98892B
:101CC100BBAA6372405125340617EFFECCDDA9B8DB
:101CD1008A9B7362504135241607FFEEDCCDB9A80B
:101CE1009A8B8495A7B6C2D3E1F008192B3A4E5FBF
:101CF1006D7C9485B7A6D2C3F1E018093B2A5E4FEB
:101D01007D6CA5B48697E3F2C0D129380A1B6F7E9A
:101D11004C5DB5A49687F3E2D0C139281A0B7F6ECA
:101D21005C4DC6D7E5F48091A3B24A5B69780C1D7E
:101D31002F3ED6C7F5E49081B3A25A4B79681C0DAA
:101D41003F2EE7F6C4D5A1B082936B7A48592D3C5A
:101D51000E1FF7E6D4C5B1A092837B6A58493D2C8A
:101D61001E0F0089129B24AD36BF48C15AD36CE5C2
:101D71007EF78108931AA52CB73EC940DB52ED646A
:101D8100FF76028B109926AF34BD4AC358D16EE756
:101D91007CF5830A9118A72EB53CCB42D950EF664A
:101DA100FD74048D169F20A932BB4CC55ED768E136
:101DB1007AF3850C971EA128B33ACD44DF56E9602A
:101DC100FB72068F149D22AB30B94EC75CD56AE316
:101DD10078F1870E951CA32AB138CF46DD54EB620A
:101DE100F97008811A932CA53EB740C952DB64ED06
:101DF10076FF89009B12AD24BF36C148D35AE56CEA
:101E0100F77E0A8318912EA73CB542CB50D966EFD5
:101E110074FD8B029910AF26BD34C34AD158E76EC9
:101E2100F57C0C851E9728A13AB344CD56DF60E9B5
:101E310072FB8D049F16A920BB32C54CD75EE168A9
:101E4100F37A0E871C952AA338B146CF54DD62EB95
:101E510070F98F069D14AB22B930C74ED55CE36A89
:101E6100F1780008040C020A060E0109050D030BA6
:101E7100070FFF1831FF1837FF183CFF1840FF18F4
:101E810046FF184BFF184EFF1851FF1855FF185900
:101E9100FF185CFF1860FF1867FF186EFF1873FFCB
:021EA1001879AE
:1050E100EF540F901E6393FEC454F0FEEFC4540FAF
:0450F100932EFF22D9
:030023000245EDA6
:0B45ED00C0E0C083C082C0D075D018B1
:1045F800309852C298755E01AF9920164820120B68
:10460800EF64027040D212D291803A301A04C21A72
:104618008024BF0904D21A802CBF0205530B808066
:1046280024BF0312906614E50BF0630B80530B80D4
:10463800C212C291800F7437250BF582E43466F5F7
:1046480083EFF0050B30992B301326906185E0FF3E
:10465800E50CC39F4008C213D21DC2908013D290AC
:10466800AF0C050C74372FF582E43467F583E0F559
:0346780099C2994B
:09467B00D0D0D082D083D0E0320F
:103C83007BFF7A18797A1223D5906EDDE070147574
:103C93002FFF7530187531EA7BFF7A1879AC122340
:103CA300D58012752FFF7530187531F97BFF7A189F
:103CB30079AC1223D57BFF7A197908906186E0F5F8
:103CC3002F1223D57BFF7A19792E906101E0F52F0E
:103CD3001223D57BFF7A197955906100E0F52F12F5
:103CE30023D57BFF7A19797BA211E433F52F1223B5
:103CF300D57BFF7A1979A41223D5752FFF75301957
:103D03007531EB7BFF7A1979D41223D5906838E0AB
:103D1300FEA3E0FFC3E49FFFE49EFEAB07FA3395E7
:103D2300E0F9F87F007E8C7D0A7C00122AF18F3245
:103D33008E318D308C2F7BFF7A1A791C1223D57B21
:103D4300FF7A1A797E906403E0F52F1223D57BFF67
:103D53007A1A7994A21EE4336401F52F1223D57BDA
:103D6300FF7A1A79ABA219E433F52F1223D57BFF1F
:103D73007A1A79D1A214E433F52F1223D57BFF7A73
:103D83001A79F7A21BE433F52F1223D57BFF7A1B95
:093D9300791F85092F1223D522A6
:1039B9007E1B7F4F1248AEEF4E70037F0122E490C9
:1039C9006EDDF07E1B7F521248AEEF4E601512502D
:1039D900C7BF3106906EDD740AF0BF3206906EDD06
:1039E9007464F07E1B7F581248AEEF4E600A124C89
:1039F900E9906186EFF080069061867402F07E1B83
:103A09007F5E1248AEEF4E600A124CE9906101EFF9
:103A1900F080069061017402F07E1B7F641248AE4B
:103A2900EF4E600A124CE9906100EFF08006906158
:103A3900007402F07E1B7F6A1248AEEF4E600D12D1
:103A49004CE9EC4D4E4F24FF92118002C2117E1BAE
:103A59007F701248AEEF4E6023124CE9A804A90505
:103A6900AA06AB077F007E8C7D0A7C00122AF11220
:103A79002B83906838EEF0A3EFF0800A90683874D1
:103A8900FFF0A374DCF07E1B7F761248AEEF4E6028
:103A99000A124CE9906403EFF08006906403740104
:103AA900F07E1B7F7C1248AEEF4E600E1250C7EFBE
:103AB90024D0640124FF921E8002C21E7E1B7F82D5
:103AC9001248AEEF4E600C1250C7EF24D024FF927B
:103AD900198002C2197E1B7F881248AEEF4E600C16
:103AE9001250C7EF24D024FF92148002C2147E1B07
:103AF9007F8E1248AEEF4E600C1250C7EF24D024CF
:103B0900FF921B8002C21B7E1B7F941248AEEF4EB0
:0E3B19006007124CE98F098003E4F5097F0074
:013B2700227B
:102F8300E4F527E52775F003A42473F582E4341EE2
:102F9300F583E493FB740193FA740293F9122A1AEA
:102FA300700302318BE4F529F52AF5287467252887
:102FB300F582E43469F583E0FF7003023186E52787
:102FC30075F003A42473F582E4341EF583E493FBC4
:102FD300740193FA740293F9852982758300122A86
:102FE30033FEEFB50608752A010529023181E52A6A
:102FF3007003023181EE600302317CE527B40F00D8
:10300300400302318690300FF828287302303C02C7
:1030130030830230BC0230C10231860231190231E1
:10302300860230EC0231860231860231460231706B
:1030330002317402318602317874672528F9E43449
:1030430069FA7B01C0031B8B32753300753400E4CE
:10305300F535D00312351D8F2E8E2D8D2C8C2BAB79
:103063002EAA2DA92CA82B7F007E8C7D0A7C001212
:103073002AF1122B83906838EEF0A3EFF002318629
:1030830074672528F582E43469F583E024D09061E0
:1030930086F074682528F582E43469F583E024D04A
:1030A300906101F074692528F582E43469F583E0C1
:1030B30024D0906100F0023186D21B0231867467FE
:1030C3002528F9E43469FA7B01C0031B8B3275337D
:1030D30000753400E4F535D00312351D8F2E8E2D87
:1030E3008D2C8C2B8F0902318674672528F9E434E3
:1030F30069FA7B01C0031B8B32753300753400E41E
:10310300F535D00312351D8F2E8E2D8D2C8C2B90E3
:103113006EDDEFF0806D74672528F9E43469FA7B7E
:1031230001C0031B8B32753300753400E4F535D0D1
:103133000312351D8F2E8E2D8D2C8C2B906403EF57
:10314300F0804074672528F9E43469FA7B01C003F1
:103153001B8B32753300753400E4F535D00312351B
:103163001D8F2E8E2D8D2C8C2BD21E8016D211806E
:1031730012D214800EC219800AE4F52AF529052813
:08318300022FAF0527022F8681
:01318B002221
:10337500C229C21CC218C217C215E4906837F0C230
:103385001F9066167405F0C22BE4F508FF7F409088
:1033950061B9E4F0A3DFFCE4FF7F20906617E4F059
:1033A500A3DFFCE4FF74042FF582E43466F583E4BF
:1033B500F0740C2FF582E43466F583E4F00FBF0852
:1033C500E4E4F50DF50EF512F511906302F0906346
:1033D50001F0C213C21DC216C212C21AF50C9061C9
:1033E50085F0F509F50BF55EC210C21B90683874BF
:1033F500FFF0A374F4F0E4906403F0C21EC211C29E
:1034050014D219906EDDF01239B9EF6003122F83D3
:10341500E4F5137E617F87906186E0F513E513C3BC
:1034250094014007E513D394084003E4F513E5132D
:1034350060220FEFAC0670010E14F5828C8374C404
:10344500F015130FEFAC0670010E14F5828C83E5B1
:1034550013F080DA906101E0F513E513C3940140A0
:1034650007E513D394084003E4F513E51360220F31
:10347500EFAC0670010E14F5828C8374C8F0151339
:103485000FEFAC0670010E14F5828C83E513F08006
:10349500DA906100E0F513E513C394014007E513E5
:1034A500D394084003E4F513E51360220FEFAC064F
:1034B50070010E14F5828C8374C2F015130FEFACF6
:1034C5000670010E14F5828C83E513F080DA0FEF98
:1034D500AC0670010E14F5828C83E4F08F828E8326
:1034E500F0F513C2ADF5C9D2CDD2CCC2C9C2CAF569
:1034F500CDF5CC906838E0F5CBA3E0F5CA85CBCD0A
:1035050085CACCD29ED29CD2CAC2ACC298C2997589
:07351500B81075B710D2AC2D
:01351C00228C
:1050F500E5106FFF901D6393650FF510EF901C632E
:0351050093F50F10
:015108002284
:0243EA008F2D15
:1043EC00E4FC752E61752F02F510F50FFDEDC395EC
:1043FC002D5017052FE52FAE2E7002052E14F582C9
:10440C008E83E0FF1250F50D80E3052FE52FAE2EC5
:10441C007002052E14F5828E83E510F0852F8285AF
:10442C002E83E50FF0052D052D7E677F37752E61E8
:10443C00752F028F828E837402F00FBF00010E0C59
:10444C00E4FDEDC3952D5038852F82852E83E0F940
:10445C0064026008E964036003B9090D8F828E83DE
:10446C007409F00FBF00010E0C8F828E83E9F00FE0
:10447C00BF00010E0C052FE52F7002052E0D80C21A
:0F448C008F828E837403F00FBF00010E0CAF04FC
:01449B0022FE
:03515300C216225F
:104ECA008F2C201335AF2C1243EA906185EFF02026
:104EDA000B127E1B7F9A123FA77E617F02E4FBAD15
:104EEA002C124170301B057F0112513DE509600308
:0B4EFA00F55B22E4F50CD213D29922E4
:022CE0008F283B
:102CE200E54724BE7003022F2B24FA7003022EA3A1
:102CF20024046003022F82E54830E703022DA73047
:102D02000C077E1B7FA6123FA7E54A6068E549C310
:102D120094024003022F82E5497007E54A14F5291F
:102D22008006E54A241FF529E52975F004A4240349
:102D3200F582746335F0F5837D4C7F04123255E5DC
:102D42002975F004A42401F582746235F0F5837DBF
:102D5200507F0412325574F92549F582E43461F545
:102D6200837481F074B92529F582E43461F58374A2
:102D720001F0D21722300C077E1B7FB1123FA774DD
:102D8200042549F582E43466F5837401F0E549755A
:102D9200F004A42417F582746635F0F5837D4C7F28
:102DA2000412325522E54B64086003022F82E54982
:102DB200C394044003022F82300C077E1B7FBB1298
:102DC2003FA7752801E54A5407FFE528A8070880B0
:102DD20002C333D8FCF5287408250EF50EB50D068E
:102DE2007408250DF50DE54A547FFFE549C43354B7
:102DF200E02FFE7400250EF582E43460F583EEF0D8
:102E0200E54AC394805022EF131313541FFFE54980
:102E120025E025E02F2417F582E43466F583E0FFF0
:102E2200E528F4FEEF5EF0802EE54A547FFF13138F
:102E320013541FFFE54925E025E02F2417F582E40E
:102E42003466F583E04528F07400250EF582E434FB
:102E520060F583E04480F07401250EF582E434606D
:102E6200F5837D4C7F04123255E551FEE550FF7C1F
:102E7200007D0A122A60EF7405250EF582E43460A3
:102E8200F583EFF07406250EF582E43460F583E5F0
:102E920052F07407250EF582E43460F583E553F0B1
:102EA20022300C077E1B7FBF123FA7E54A54E06425
:102EB200407003022F82E54A547FF529E549701DCF
:102EC200E5291313543FFF7401A807088002C33396
:102ED200D8FC4211906301E04511F08024E5496479
:102EE200016003022F82E5291313543FFF7401A8E6
:102EF20007088002C333D8FC4212906302E04512F5
:102F0200F0E54975F020A47C002529FFEC35F0FEA0
:102F1200EF25E0FFEE33FE74042FF58274643EF574
:102F2200837D4CAF4B12325522E54AB40113300C6B
:102F3200077E1B7FC4123FA7E54D04906FF6F0C2D7
:102F420029E54AB40216240CF582E43466F583E5D9
:102F52004DF0300C077E1B7FCB123FA7E54AB4032E
:102F62001F240CF582E43466F583E54DF0300C073E
:102F72007E1B7FD4123FA7302906906FDE7402F0C9
:012F8200222C
:10090200906403E070030211BD30002F050A906667
:1009120016E0600214F0906837E0600214F0C20042
:10092200302918906184E004F0E0D3940A400C303E
:100932000C077E1B7FDC123FA7C229E55BB40109CD
:10094200E4F55BF50CD213D29930130DE50AD3947A
:10095200064009C213D21D8003E4F50A301D0AC203
:100962001D301B05E4FF12513D301303020E19E541
:100972005B6003020E19201E06201503020E19C227
:1009820015301F29C21FE4906102F0A37408F09091
:100992006403E0906104F0906615E0906105F0A3B5
:1009A20074FEF0A3748FF07F06124ECA22906FF687
:1009B200E0FF6025E4906102F0A37408F090640304
:1009C200E0906104F0A37483F0A3EFF0E4A3F0904D
:1009D2006FF6F07F06124ECA22E50E650D70030215
:1009E2000ADC906837E06003020BB6E50D2408F5D7
:1009F20028E4906102F0A37408F0906403E090612F
:100A020004F0A374F0F0A37406F0A37491F07406DA
:100A12002528F582E43460F583E0906108F07407DC
:100A22002528F582E43460F583E0906109F07401D1
:100A32002528F582E43460F583E090610AF07402BF
:100A42002528F582E43460F583E090610BF07403AD
:100A52002528F582E43460F583E090610CF074049B
:100A62002528F582E43460F583E090610DF074008E
:100A72002528F582E43460F583E0FF547FFEC394B9
:100A820040500BEFC454F00490610EF080167400D5
:100A92002528F582E43460F583E0FFC454F0240590
:100AA20090610EF074002528F582E43460F583E04D
:100AB200FFEEC4540F90610FF0EF5480FF740525D0
:100AC20028F582E43460F583E02F906110F090689D
:100AD200377414F07F0F124ECA2230186AE4906104
:100AE20002F0A37408F0906403E0906104F0A37430
:100AF20041F0A37420F0752A61752B07E4F5287480
:100B0200172528F582E43466F583E0F529301906C5
:100B1200FF1250E18F29852B82852A83E529F0F483
:100B2200FFE5822408F582E43583F583EFF0052B97
:100B3200E52B7002052A0528E528C3940840C07FEA
:100B420015124ECAC21822301C6AE4906102F0A348
:100B52007408F0906403E0906104F0A37445F0A37C
:100B62007420F0752A61752B0775280874172528DB
:100B7200F582E43466F583E0F529301906FF125058
:100B8200E18F29852B82852A83E529F0F4FFE5820E
:100B92002408F582E43583F583EFF0052BE52B700D
:100BA20002052A0528E528C3941040C07F15124E7D
:100BB200CAC21C22201703020CB99061FAE0FF900E
:100BC20061F9E04F5401D394005003020CB9E4F5EB
:100BD2002874B92528F582E43461F583E0700302B4
:100BE2000CAB74B92528F582E43461F583E4F09006
:100BF2006102F0A37408F0906403E0906104F0A332
:100C020074F0F0A37403F0A37491F0E528C4540FB8
:100C12002408A3F0E528540FA3F0E52825E025E0F9
:100C2200F5282401F582E43462F583E090610AF04C
:100C320074022528F582E43462F583E090610BF0BA
:100C420074032528F582E43462F583E090610CF0A8
:100C520074042528F582E43462F583E090610DF096
:100C6200E4A3F074032528F582E43463F583E0906D
:100C7200610FF074042528F582E43463F583E09073
:100C82006110F074052528F582E43463F583E09061
:100C92006111F074062528F582E43463F583E0904F
:100CA2006112F07F11124ECA220528E528C3944032
:100CB2005003020BD3C217906616E0704130143E07
:100CC2007478F0E4906102F0A37408F0906403E099
:100CD200906104F0A374F0F0E4A3F0A37490F0A385
:100CE2007408F0E4A3F0A3F0A3F0A3F0A3F0A3F040
:100CF200A3F0A3F0A3F0A3F07F11124ECA22E508DD
:100D0200C39404506FE50825E0FF7403A807088028
:100D120002C333D8FCF528551165287053E528F431
:100D22005211E4906102F0A37408F0906403E09021
:100D32006104F0A374F0F0A37402F0A37491F0E5DF
:100D4200082420A3F0E50833333354F875F002A4E5
:100D52002404F582E5F03464F58363A2019061090D
:100D620063A2017F101232677F17124ECA05082252
:100D72000508808AE508C394085076E50824FC2516
:100D8200E0FF7403A807088002C333D8FCF5285596
:100D92001265287058E528F45212E4906102F0A31B
:100DA2007408F0906403E0906104F0A374F0F0A37F
:100DB2007402F0A37491F0E50854032440A3F0E513
:100DC2000833333354F875F002A42404F582E5F0B5
:100DD2003464F58363A20190610963A2017F10125A
:100DE20032677F17124ECA0508530807220508808A
:100DF20083E4F508201E20E4906102F0A37408F059
:100E0200906403E0906104F0A37490F0E4A3F0A373
:100E1200F07F06124ECA22906614E0FF70030211A0
:100E2200BDF529E4F0200B1F7E1B7FEA123FA7E5E8
:100E32002954802437F582E43466AF82FEE52954D2
:100E42007FFDE4FB124170E52970030211BDE52923
:100E52005480FF2437F582E43466AD82F52A8D2B67
:100E6200E4F510F50F8F28E528C395295018052BB6
:100E7200E52BAE2A7002052A14F5828E83E0FF125A
:100E820050F5052880E1E50F4510600E300B030296
:100E920011BD7E1B7FF3123FA722E5295480243720
:100EA200F582E43466AF82F52A8F2B7402252BF586
:100EB2002BE4352AF52A852B82F583E0FF90640323
:100EC200E0FEEF6E600E300B030211BD7E1B7FFD54
:100ED200123FA722052BE52B7002052AF582852AEF
:100EE20083E0FFB43003D21522EF640170030211D4
:100EF200BDEF64187037906605E0FF906604E04F1E
:100F0200600CD218200B077E1C7F0E123FA7906642
:100F120007E0FF906606E04F70030211BDD21C305D
:100F22000B030211BD7E1C7F17123FA722852B8265
:100F3200852A83E0B41915200B077E1C7F20123FFF
:100F4200A7906301E0F511A3E0F51222852B8285BB
:100F52002A83E0FF54F064F06003021045906615A6
:100F6200EFF0052BE52B7002052AF582852A83E036
:100F7200FF64807033052BE52B7002052AF582850C
:100F82002A83E0644060030211BDD21F052BE52BCA
:100F92007002052AF582852A83E064086003021143
:100FA200BDD214906616F022EFB40127052BE52B73
:100FB2007002052AF582852A83E0644F60030211DC
:100FC200BD906837E070030211BD7408250DF50D60
:100FD200E4F022852B82852A83E060030211BD059D
:100FE2002BE52B7002052AF582852A83E064426094
:100FF200030211BD052BE52B7002052AF582852A15
:1010020083E0906FE0F0052BE52B7002052AF58254
:10101200852A83E0906FE1F0052BE52B7002052A0B
:10102200F582852A83E0906FE2F0052BE52B7002B2
:10103200052AF582852A83E0906FE3F0D22BC21451
:10104200D21F22852B82852A83E0FF64116008EF7C
:101052006412600302119BE529547F640E6003024F
:10106200119B200B077E1C7F29123FA730290E30CF
:101072000B030211BD7E1C7F3E123FA722852B82ED
:10108200852A83E0540314F529052BE52B7002050C
:101092002AF582852A83E0F52830E709E4906FDF9C
:1010A200F0906FE4F0E52830E60BE4906FDFF0900B
:1010B2006FE47410F0E52830E50B906FDF7401F0F7
:1010C200E4906FE4F0E52830E40C906FDF7401F0F7
:1010D200906FE47410F0E52830E30B906FDF740238
:1010E200F0E4906FE4F0E52830E20C906FDF7402D8
:1010F200F0906FE47410F0E52830E10B906FDF742C
:1011020003F0E4906FE4F0E52830E00C906FDF74B8
:1011120003F0906FE47410F07402252BF52BE43584
:101122002AF52A852B82F583E0F52830E700E528A9
:1011320030E607906FE4E02402F0E52830E50790FE
:101142006FE4E02404F0E52830E407906FE4E02443
:1011520006F0E52830E307906FE4E02408F0E52884
:1011620030E207906FE4E0240AF0E52830E10790CE
:101172006FE4E0240CF0E52830E007906FE4E0240F
:101182000EF0906FE4E02529F0D229E4906184F01A
:10119200906FDEF0906FF6F022200B1F7E1C7F4CCA
:1011A200123FA7E52954802437F582E43466AF82E2
:0B11B200FEE529547FFDE4FB124170B4
:0111BD00220F
:104720000211BEE493A3F8E493A34003F68001F2E0
:1047300008DFF48029E493A3F85407240CC8C3339A
:10474000C4540F4420C8834004F456800146F6DF69
:10475000E4800B0102040810204080905146E47E62
:10476000019360BCA3FF543F30E509541FFEE4935E
:10477000A360010ECF54C025E060A840B8E493A325
:10478000FAE493A3F8E493A3C8C582C8CAC583CA50
:10479000F0A3C8C582C8CAC583CADFE9DEE780BE08
:01514C000062
:102A1A00BB010689828A83E0225002E722BBFE02BA
:092A2A00E32289828A83E49322ED
:102A3300BB010CE58229F582E5833AF583E0225058
:102A430006E92582F8E622BBFE06E92582F8E222A2
:0D2A5300E58229F582E5833AF583E49322BC
:102A6000BC000BBE0029EF8DF084FFADF022E4CC5A
:102A7000F875F008EF2FFFEE33FEEC33FCEE9DEC23
:102A8000984005FCEE9DFE0FD5F0E9E4CEFD22ED69
:102A9000F8F5F0EE8420D21CFEADF075F008EF2FB3
:102AA000FFED33FD4007985006D5F0F222C398FDA4
:052AB0000FD5F0EA2241
:102AB50075F008758200EF2FFFEE33FECD33CDCCD8
:102AC50033CCC58233C5829BED9AEC99E58298405B
:102AD5000CF582EE9BFEED9AFDEC99FC0FD5F0D638
:102AE500E4CEFBE4CDFAE4CCF9A88222B800C1B962
:102AF5000059BA002DEC8BF084CFCECDFCE5F0CBA0
:102B0500F97818EF2FFFEE33FEED33FDEC33FCEBD8
:102B150033FB10D703994004EB99FB0FD8E5E4F993
:102B2500FA227818EF2FFFEE33FEED33FDEC33FC80
:102B3500C933C910D7059BE99A4007EC9BFCE99A74
:102B4500F90FD8E0E4C9FAE4CCFB2275F010EF2FB9
:102B5500FFEE33FEED33FDCC33CCC833C810D707B9
:102B65009BEC9AE899400AED9BFDEC9AFCE899F8F4
:0E2B75000FD5F0DAE4CDFBE4CCFAE4C8F92287
:0E2B8300C3E49FFFE49EFEE49DFDE49CFC2263
:102B9100EB9FF5F0EA9E42F0E99D42F0E89C45F09A
:012BA1002211
:0C2BA200ECF0A3EDF0A3EEF0A3EFF022A6
:102BAE00A8828583F0D083D082122BC5122BC5123A
:102BBE002BC5122BC5E473E493A3C583C5F0C5835F
:102BCE00C8C582C8F0A3C583C5F0C583C8C582C871
:012BDE0022D4
:10237300E53B242FF8E6053B22782C302702782F03
:10238300E475F001122C40022A1A2020EB7F2ED292
:10239300208018EF540F2490D43440D4FF30240B02
:1023A300EF24BFB41A0050032461FFE53C6002151B
:1023B3003C053FE53F7002053E30270D782CE47560
:1023C300F001122C40EF022BDF024DFC7403D227E5
:1023D3008003E4C227F53B8B2C8A2D892EE4F53C40
:1023E300F53EF53FE53C60077F201223AE80F5758F
:1023F3003DFFC221C220C222C223C225C226C22857
:1024030012237CFF700D3027057F001223BFAF3FDF
:10241300AE3E22B4255FC2D5C22412237CFF24D052
:10242300B40A00501A75F00A783C30D50508B6FF97
:102433000106C6A426F620D5047002D22380D9242F
:10244300CFB41A00EF5004C2E5D2240225BFD22133
:1024530080C6D22080C0D22280BCD2D580BAD225F9
:1024630080B47F201223AE2022077401B53C0040C4
:10247300F1122373FF1223AE0223E7D228D2268060
:1024830095122373FB122373FA122373F94A4B70C9
:102493000679907A267BFF20222EE53C602A7E0077
:1024A3008E82758300122A3360060EEE653D70F04E
:1024B300C2D5EBC0E0EAC0E0E9C0E0EE122606D0E8
:1024C300E0F9D0E0FAD0E0FB122A1AFF60AAEBC0D1
:1024D300E0EAC0E0E9C0E01223AED0E02401F9D085
:1024E300E03400FAD0E0FBE53D0460DCD53DD98063
:1024F300877BFF7A267902D222809C791080027929
:1025030008C226C2288008D2D5790A8004790AC273
:10251300D5E53D047002F53DE4FAFDFEFF12237399
:10252300FC7B08202113122373FD7B1030200A1239
:102533002373FE122373FF7B20EC3382D592D55095
:1025430013C3E43020069FFFE49EFEE42021039D95
:10255300FDE49CFCE4CBF8C221EC700CCFCECDCCD7
:10256300E824F8F870F38017C3EF33FFEE33FEED82
:1025730033FDEC33FCEB33FB994002FB0FD8E9EB63
:10258300302105F8D0E0C448B221C0E00AEC4D4E3A
:102593004F78207B0070C2EAB53D0040BCC0E0121A
:1025A3002608D0F0D0E0202104C4C0E0C4B221C08A
:1025B300F0122397D0F0D5F0EB0223E7122C9F24DF
:1025C300845324FE5824554C24514225024F250A96
:0F25D30044250A49246A4325105524F44624F46C
:1025E2004524F44726B05024592D245D2E24802BF7
:1025F200246123247E2026992A2419480000247865
:102602003F3F3F00790AA2D5202314302509B91093
:10261200020404B9080104A2D520260250010420B4
:1026220022689222B53C005034C0E07F203023194A
:102632007F30A22272267225500F12265FC222C25A
:1026420026C225C2287F30800F302503E9C0E01260
:1026520023AE302503D0E0F9D0E0B53CCC302517CD
:102662007F30B9100C1223AE7F583024077F788058
:1026720003B908031223AE3022057F2D0223AE7F59
:10268200202028F87F2B2026F322922280CF286E4A
:10269200756C6C2900D2211223733021F8C2217883
:1026A2003C30D50108F60224192D50434958122313
:1026B200732403B405004001E49026AB9312239FD8
:0D26C200743A12239FD223753C040224FEBB
:10351D008B2F8A308931E4F53BF53AF539F538F5DD
:10352D0036F537E533453445326012EBC0E0EAC07D
:10353D00E0E9C0E0AB32AA33A934122C50AB2F0511
:10354D0031E531AA307002053014F9122A1AF53C12
:10355D00C394094007E53CD3940D40E1E53C64205C
:10356D0060DBE53CB42D054337038016E53CB42BF9
:10357D0005433701800C74FF2531F53174FF35306B
:10358D00F530E53560046410703FAB2FAA30A931DA
:10359D00122A1A64306009E535702E75350A8029B6
:1035AD00900001122A33FF64786004EFB45813437E
:1035BD00370175351074022531F531E43530F530AC
:1035CD008007E5357003753508AB2F0531E531AA58
:1035DD00307002053014F9122A1AF53CC39461407B
:1035ED000AE53CD3947A5003533CDF74D0253CF567
:1035FD003CC3940A400CE53C9411406D74F9253C94
:10360D00F53CE53CD395355060433701853B40850E
:10361D003A3F85393E85383DAF357E00E4FCFDAB44
:10362D003BAA3AA939A838122BF1C8ECC8C9EDC983
:10363D00CAEECACBEFCBE4FCFDFEEB253CF53BEE31
:10364D003AF53AED39F539EC38F538AF3BAE3AADE0
:10365D0039FCAB40AA3FA93EA83DD3122B91500394
:10366D000235D64337040235D6E53720E003E48032
:10367D002DE53345344532601EAB2FE53124FFF97E
:10368D00E53034FFFAEBC0E0EAC0E0E9C0E0AB3270
:10369D00AA33A934122C50E53730E20774FFFFFE30
:1036AD00FDFC22E537AF3BAE3AAD39AC3830E10326
:0436BD00022B832237
:102BDF00BB010689828A83F0225002F722BBFE01D5
:022BEF00F322CF
:102BF100E88FF0A4CC8BF0A42CFCE98EF0A42CFC83
:102C01008AF0EDA42CFCEA8EF0A4CDA8F08BF0A400
:102C11002DCC3825F0FDE98FF0A42CCD35F0FCEB5F
:102C21008EF0A4FEA9F0EB8FF0A4CFC5F02ECD3924
:0F2C3100FEE43CFCEAA42DCE35F0FDE43CFC2291
:102C4000FAE6FB0808E6F925F0F618E6CA3AF62295
:102C5000BB011A89828A83D0F0D0E0F8D0E0F9D0A5
:102C6000E0FAD0E0FBE8C0E0C0F0022CCE5016E95C
:102C7000F8D083D082D0E0F9D0E0FAD0E0FBC08277
:102C8000C083022CC5BBFE16E9F8D083D082D0E009
:0F2C9000F9D0E0FAD0E0FBC082C083022CD7223B
:102C9F00D083D082F8E4937012740193700DA3A3C4
:102CAF0093F8740193F5828883E4737402936860D8
:062CBF00EFA3A3A380DFD8
:092CC500EBF608EAF608E9F62234
:092CCE00EBF0A3EAF0A3E9F02207
:092CD700EBF208EAF208E9F2222E
:00000001FF
